:100000000C9455060C949C060C949C060C949C062F
:100010000C949C060C949C060C949C060C949C06D8
:100020000C949C060C949C060C9472150C9444162B
:100030000C94D7240C949C060C949C060C949C065F
:100040000C949C060C949C060C949C060C949C06A8
:100050000C949C060C9477250C949C060C949C069E
:100060000C949C060C94E9080C949C060C949C0639
:100070000C949C060C949C060C949C060C949C0678
:100080000C949C060C949C060C949C060C949C0668
:100090000C949C060C949C060C949C060C949C0658
:1000A0000C949C060C949C060C949C06150E190E40
:1000B0001D0E210E250E290E2D0E310E350E390E78
:1000C0003D0E410E450E490E4D0E510E550E590E68
:1000D0005D0E610E650E690E6D0E710E750E790E58
:1000E0007D0E810E850E890E8D0E910E950E990E48
:1000F0009D0EA10EE10E130EA50EA70EA90EAB0EBE
:10010000AF0EB30EB70EBB0EC00EC50EC90ECD0E90
:10011000D10ED50ED90EDF0EDF0EDF0EDF0EDF0E95
:10012000DF0EDF0EDF0EDF0EDF0EDF0EDF0EDF0E67
:10013000DF0EDF0EDF0EDF0EDF0EDF0EDD0EB1167F
:10014000D316C117D316C11718173B17C11790172D
:10015000A317CB1ACB1AFA1AFA1A581B961BB01D02
:10016000B01DAF1BB01DB01CB01C841DB01DB01D58
:100170009B1D1F141A16041D1B06202115080709B4
:10018000190522231C170A0B11801E352B39797A89
:100190007B2C2425180C0E0D1080742A31287C7DB0
:1001A0007E7F26271213330F36802D2E302F3438C2
:1001B000378025630025730D0A00522C310D0A008B
:1001C00053592C464646340D0A0053482C303033E0
:1001D000430D0A00537E2C360D0A0053572C38303D
:1001E00030300D0A00534D2C340D0A0053532C4B64
:1001F0006579626F6172642F4D6F7573650D0A00CA
:10020000532D2C546D6B42540D0A0053462C310D66
:100210000A002D2D2D0D0A0045786974696E67203E
:10022000636F6E666967206D6F6465202E2E2E0ADF
:10023000002B0D0A00760D0A0024242400456E745C
:100240006572696E6720636F6E666967206D6F64A3
:1002500065202E2E2E0A00522C310D0A0053522CEE
:100260005A0D0A00555342206D6F64650A004175AE
:10027000746F206D6F64650A00253032750A0025A1
:100280003032753A00253032753A004241543A20F6
:1002900025756D560900757074696D653A202530B5
:1002A000327520253032753A253032753A25303294
:1002B000750A00564255533A2025580A0052656D7A
:1002C0006F746557616B657570456E61626C6564CE
:1002D0003A2025580A000A003F004C4F5700444975
:1002E000534348470043484152470046554C4C0051
:1002F000626174746572793A2000555342205374D8
:100300006174653A2025730A00636F6E6669675FE2
:100310006D6F64653A2025580A00726E34325F6151
:1003200075746F636F6E6E656374696E6728293AC2
:100330002025580A00726E34323A2025730A00666E
:100340006F7263655F7573623A2025580A00707298
:100350006F746F636F6C3A2025730A000A2D2D2D80
:100360002D2D20524E2D343220696E666F202D2D9A
:100370002D2D2D0A00753A20202020202020746F7A
:1003800067676C6520466F72636520555342206D28
:100390006F64650A00703A202020202020207061C0
:1003A0006972696E670A00536C636B3A20202020E3
:1003B000524E2D343220696E697469616C697A65B8
:1003C0000A0044656C3A2020202020656E74657216
:1003D0002F6578697420524E2D343220636F6E661B
:1003E0006967206D6F64650A00623A202020202032
:1003F00020206261747465727920766F6C74616715
:10040000650A00693A20202020202020524E2D34F9
:100410003220696E666F0A000A0A2D2D2D2D2D20BF
:10042000426C7565746F6F746820524E2D343220A3
:1004300048656C70202D2D2D2D2D0A00253032752C
:100440003A253032753A253032750925756D560AD0
:10045000004C4544207374617475733A2025303222
:10046000580A002025303258002563005B735D0078
:100470004B6579626F6172642073746172740A00F3
:10048000524E2D343220696E69740A000A55534267
:1004900020696E69740A005B445D005B435D001275
:1004A00003480048004B00420020006D006F0064CC
:1004B0000000000E0374002E006D002E006B002E55
:1004C0000000000403090409027400040100A032C2
:1004D00009040000010301010009211101000122AA
:1004E00040000705810308000A0904010001030117
:1004F0000200092111010001224D000705820308B5
:10050000000A090402000103000000092111010092
:10051000012236000705830308000A0904030002CC
:1005200003000000092111010001222200070584B7
:10053000032000010705040320000112011001003F
:10054000000008EDFE42420401010200010631FFF5
:100550000974A1010975150026FF00952075088111
:10056000020976150026FF00952075089102C00546
:10057000010980A101850216810026B7001A8100B9
:100580002AB700751095018100C0050C0901A10171
:100590008503160100269C021A01002A9C02751090
:1005A00095018100C005010902A1010901A1000511
:1005B0000919012905150025019505750181029587
:1005C00001750381010501093009311581257F95E8
:1005D000027508810609381581257F950175088106
:1005E00006050C0A38021581257F950175088106DC
:1005F000C0C005010906A101050719E029E715009A
:10060000250195087501810295017508810105088C
:10061000190129059505750191029501750391014F
:100620000507190029FF150026FF009506750881AA
:1006300000C0636F6E73756D65723A202530345853
:100640000A0073797374656D3A20253034580A00B6
:100650000A002530325820006B6579626F61726440
:100660003A20004C45443A20253032580A002530C3
:1006700032583A202530386225730A00722F6320E1
:1006800030313233343536370A004F6E6573686F58
:10069000743A2074696D656F75740A00290A002523
:1006A00075002F002575005D2800256400200025B9
:1006B0006400200025640020002564007C002530B3
:1006C0003258006D6F7573656B6579205B62746E6F
:1006D0007C782079207620685D287265702F6163B0
:1006E0006C293A205B006D6B5F776865656C5F74A1
:1006F000696D655F746F5F6D6178203D2025640AC8
:10070000006D6B5F776865656C5F6D61785F7370B6
:10071000656564203D2025640A006D6B5F74696D1A
:10072000655F746F5F6D6178203D2025640A006D00
:100730006B5F6D61785F7370656564203D20256433
:100740000A006D6B5F696E74657276616C203D2086
:1007500025640A006D6B5F64656C6179203D20251E
:10076000640A006D6B5F776865656C5F74696D65C1
:100770005F746F5F6D6178203D2025640A006D6BAA
:100780005F776865656C5F6D61785F7370656564E0
:10079000203D2025640A006D6B5F74696D655F7490
:1007A0006F5F6D6178203D2025640A006D6B5F6D81
:1007B00061785F7370656564203D2025640A006D73
:1007C0006B5F696E74657276616C203D2025640AEA
:1007D000006D6B5F64656C6179203D2025640A00C3
:1007E0000A00257500363A20776865656C5F746984
:1007F0006D655F746F5F6D61783A20000A00257542
:1008000000353A20776865656C5F6D61785F73705D
:100810006565643A20000A00257500343A20746941
:100820006D655F746F5F6D61783A20000A00257511
:1008300000333A206D61785F73706565643A20001B
:100840000A00257500323A20696E74657276616C13
:10085000286D73293A20000A00257500313A20647A
:10086000656C6179282A31306D73293A20000A09B4
:100870002D2056616C756573202D0A004D3E004D8C
:1008800025643E20003F00736574206465666175D1
:100890006C740A00433E20007768657265206465C9
:1008A0006C74613A20637572736F723D25642C20FD
:1008B000776865656C3D25640A53656520687474C6
:1008C000703A2F2F656E2E77696B69706564696168
:1008D0002E6F72672F77696B692F4D6F7573655F28
:1008E0006B6579730A000A092D204D6F7573656B6E
:1008F0006579202D0A4553432F713A097175697442
:100900000A313A0964656C6179282A31306D73299E
:100910000A323A09696E74657276616C286D7329C2
:100920000A333A096D61785F73706565640A343A19
:100930000974696D655F746F5F6D61780A353A0996
:10094000776865656C5F6D61785F73706565640A73
:10095000363A09776865656C5F74696D655F746FB9
:100960005F6D61780A0A703A097072696E74207658
:10097000616C7565730A643A097365742064656611
:1009800061756C74730A75703A092B310A646F775C
:100990006E3A092D310A706775703A092B31300AA9
:1009A0007067646F776E3A092D31300A0A7370658B
:1009B0006564203D2064656C7461202A206D617837
:1009C0005F7370656564202A2028726570656174A4
:1009D000202F2074696D655F746F5F6D6178290ADF
:1009E000003F004D3E2000433E20004C25640A009D
:1009F0000A092D20436F6E736F6C65202D0A4553D5
:100A0000432F713A09717569740A6D3A096D6F75F2
:100A100073656B65790A000A092D204D616769636A
:100A2000202D0A643A0964656275670A783A096498
:100A300065627567206D61747269780A6B3A096442
:100A400065627567206B6579626F6172640A6D3AE1
:100A5000096465627567206D6F7573650A763A097A
:100A600076657273696F6E0A733A0973746174758F
:100A7000730A633A09636F6E736F6C65206D6F6400
:100A8000650A302D343A096C61796572302D34284D
:100A90004631302D4634290A506175733A09626F28
:100AA0006F746C6F616465720A003F0074696D65F4
:100AB000725F72656164333228293A202530346CC4
:100AC000580A006B6579626F6172645F69646C6576
:100AD0003A2025580A006B6579626F6172645F7015
:100AE000726F746F636F6C3A2025580A00686F73D9
:100AF000745F6B6579626F6172645F6C65647328A3
:100B0000293A2025580A000A092D2053746174756A
:100B100073202D0A004743433A20342E392E3220C9
:100B20004156522D4C4942433A20312E382E3073D3
:100B3000766E204156525F415243483A20617672A8
:100B4000350A004F5054494F4E533A204C554641B8
:100B5000204D4F5553454B45592045585452414B14
:100B6000455920434F4E534F4C4520434F4D4D4127
:100B70004E44204B45594D41505F53454354494FD6
:100B80004E20343039360A004255494C443A20341C
:100B90003139303537312D64697274792028303716
:100BA0003A35353A3531204F6374203238203230AF
:100BB0003137290A005649443A20307846454544A1
:100BC00028742E6D2E6B2E29205049443A203078FF
:100BD000343234322848484B42206D6F6429205605
:100BE00045523A203078303130340A00444553437E
:100BF0003A20742E6D2E6B2E206B6579626F6172B8
:100C000064206669726D7761726520666F72204834
:100C1000484B42206D6F640A000A092D2056657208
:100C200073696F6E202D0A000A6D6F7573653A2027
:100C30006F66660A000A6D6F7573653A206F6E0AFB
:100C4000000A6B6579626F6172643A206F66660AAA
:100C5000000A6B6579626F6172643A206F6E0A00F8
:100C60000A6D61747269783A206F66660A000A6DCF
:100C700061747269783A206F6E0A000A6465627561
:100C8000673A206F6E0A000A64656275673A206FE2
:100C900066660A000A0A626F6F746C6F616465723F
:100CA0002E2E2E2000433E20000011241FBECFEF29
:100CB000DAE0DEBFCDBF04B603FE27C080919F03FC
:100CC0009091A003A091A103B091A2038730904B13
:100CD000A740B04BD1F410929F031092A003109242
:100CE000A1031092A20314BE84B7877F84BF0FB6FE
:100CF000F894A895809160008861809360001092BC
:100D000060000FBEE0E0F8E3099511E0A0E0B1E07B
:100D1000E0E0FCE502C005900D92AA39B107D9F7D1
:100D200023E0AAE9B1E001C01D92AF39B207E1F7B3
:100D30000E941C100C94FE2D0C9400000FB68095A0
:100D40009AE0F8947BE27A95F1F708F0589A08F463
:100D5000589886959A95B1F70FBE08950FB680E81A
:100D6000F894499BFECF4999FECF96E19A95F1F709
:100D70009CE29A95F1F7869549998068C8F70FBE6D
:100D800008950FB680E8F89496E19A95F1F79CE201
:100D90009A95F1F7869549998068C8F796E19A95F2
:100DA000F1F7499BFECF0FBE0895FF93EF93E091BB
:100DB0009A01F0919B01309709F00995EF91FF910D
:100DC0000895FC018591803011F0EFDFFBCF08958D
:100DD000FF27E0E230E247FF0CC0419597FF09C0D2
:100DE000EDE26095709580959095611D711D811D56
:100DF000911D27FF02C0219530E350E2AA27660F1C
:100E0000771F881F991FAA1FA41710F0A41B6395B2
:100E10005A95A9F7AA3008F0A95FA05DAF93F395A2
:100E2000611571058105910541F7ED3211F4EF93DC
:100E3000F395F21718F43F93F395FBCF8F91B5DF3D
:100E4000FA95E1F70895E991F9918591803021F0C3
:100E5000853219F0AADFF9CF089520E0E894559182
:100E60005532C1F3503311F4689455915A3348F414
:100E7000505390F3220F022E220F220F200D250F28
:100E8000F4CF0EF4219589919991533619F3533784
:100E900029F1533559F1BC0188279927E8945C362C
:100EA00021F48991999168945591543639F446EF1B
:100EB0007EF077FF0DC08FEF9FEF0AC055374AE0F5
:100EC00039F0583540E121F0523642E009F00895FA
:100ED000FF93EF937DDFEF91FF91B7CFFF93EF93F8
:100EE000FC0181918030B9F360DFFBCFFF93EF937A
:100EF00068DFF1CFDF93CF93CDB7DEB72596A3DFC1
:100F0000CF91DF91089514B88FEF85B9549A5C980A
:100F100008958FEF84B980E485B9549A5C9A8FE183
:100F20009EE40197F1F700C0000008958FEF84B9A7
:100F300080E485B957985F9A87B18F7387B988B174
:100F4000806C88B92E9A2F980E948307E4EAF1E01A
:100F500088E08E0F11928E13FDCFECE9F1E088E06E
:100F60008E0F11928E13FDCF84EA91E09093AF0122
:100F70008093AE018CE991E09093AD018093AC0138
:100F800008950F931F93CF93DF938091AC019091BD
:100F9000AD012091AE013091AF013093AD012093AE
:100FA000AC019093AF018093AE015C9B0E948907D6
:100FB000C0E0D0E001E010E080E090E025B1207CCE
:100FC0002C2BAC0133E0440F551F3A95E1F7242B4D
:100FD00025B9EAE1EA95F1F700C0E091AC01F091A2
:100FE000AD01EC0FFD1F208130E0082E02C03595C9
:100FF00027950A94E2F720FD2F9AF5E3FA95F1F789
:101000000000E6B52E982AE12A95F1F700C040913C
:10101000AE015091AF01DA01AC0FBD1F4F9B0AC06A
:101020009801082E01C0220F0A94EAF720953C91FE
:10103000232308C06C919801082E01C0220F0A9446
:10104000EAF7262B2C9326B56E2F70E02E1718F09A
:1010500026B530E004C026B530E021503F4F261BB6
:10106000370B2630310558F0E091AC01F091AD011D
:10107000EC0FFD1F2081FA01EC0FFD1F20833AE1E8
:101080003A95F1F700C02F982E9AEBE2F1E03197F4
:10109000F1F700C0000001968830910509F08ECF6D
:1010A000A091AE01B091AF01AC0FBD1FE091AC01BA
:1010B000F091AD01EC0FFD1F9C918081981751F0CC
:1010C0000E9415256093B0017093B1018093B20125
:1010D0009093B3012196C830D10509F06DCF5C9B88
:1010E0001BC080919603853021F080919603811179
:1010F00013C06091B0017091B1018091B2019091E3
:10110000B3010E944B25613177428105910520F0A2
:101110000E9483070E94962481E0DF91CF911F9166
:101120000F9108952091AE013091AF01F901E80FC0
:10113000F11D808108950C9489070C948307569AB9
:1011400081FF02C05E9A08955E98089588E08093BA
:10115000CC001092CD00E9ECF0E0808180698083C2
:10116000808188608083EAECF0E080818083EBEC12
:10117000F0E080818083559A5D98789408959091ED
:10118000B5012091B4019217D1F030E0F901EA5491
:10119000FE4F80812F5F3F4F33272093B401492FAB
:1011A00050E0921718F4241B350B03C0241B350B99
:1011B0003395233031050CF05D9890E008958FEF62
:1011C0009FEF08959091C80095FFFCCF8093CE00CB
:1011D00008951F920F920FB60F9211242F933F93F1
:1011E0004F935F938F939F93EF93FF938091B501FC
:1011F00090E0AC014F5F5F4F2091B401241741F0A4
:101200003091CE00FC01EA54FE4F30834093B5018B
:101210003091B501822F90E0432F50E0841B950B55
:10122000321708F0939503970CF45D9AFF91EF91B4
:101230009F918F915F914F913F912F910F900FBE92
:101240000F901F9018958091D00208950895809175
:10125000D00208950895089508950895CF93DF93D7
:101260008D3C9105B9F1B8F4853B9105A9F148F49D
:10127000833B9105D1F1843B9105D1F5D0E0C0E2EB
:101280003BC0873B910571F150F18C3C910581F594
:10129000D0E0C8E031C08A3E9105C1F040F4823E02
:1012A0009105B1F0893E910519F5D0E124C0813254
:1012B00022E0920749F0833222E09207D9F08A387F
:1012C0009140B1F4D2E017C0D4E015C0D0E213C011
:1012D000D0E411C0D0E80FC0D0E0C1E00DC0D0E034
:1012E000C2E00AC0D0E0C4E007C0D0E0C0E104C062
:1012F000D0E001C0D1E0C0E08DEF0E94E20883E0C1
:101300000E94E20883E00E94E2088D2F0E94E2081A
:101310008C2FDF91CF910C94E208CF93DF93EC01F7
:101320008DEF0E94E20885E00E94E20882E00E94C0
:10133000E20888810E94E20889810E94E2088A818D
:101340000E94E2088B81DF91CF910C94E208CF9349
:10135000DF93EC018DEF0E94E20889E00E94E20831
:1013600081E00E94E20888810E94E20880E00E94F9
:10137000E2088A810E94E2088B810E94E2088C8147
:101380000E94E2088D810E94E2088E810E94E2089C
:101390008F81DF91CF910C94E2080C94BF08EF92FB
:1013A000FF920F931F93CF938C010E9409257C011C
:1013B000C0E0C7010E9421258017910798F40E9480
:1013C000BF089C012F3F8FEF380751F02D3041F0BF
:1013D0002A3041F0EC2FF0E0E854FD4F2083CF5F3E
:1013E000C73138F3EC2FF0E0E854FD4F108288EB62
:1013F00092E0CF911F910F91FF90EF9008950C9480
:10140000E20881B3881F8827881F0895879A8F9ADA
:10141000089585B7806885BF85B7806885BF0E94BD
:10142000060A86988E9A81988998559A5D980C94A8
:10143000A608879A8F9808958FB186958170089530
:101440008FB186FB882780F908958093D002089594
:10145000CF93DF93FC018491EF012196882321F043
:101460000E94E208FE01F7CFDF91CF910895CF935C
:10147000DF93C2EBD1E00E94BF088F3F2FEF9207AE
:1014800059F09F938F93DF93CF930E947A070F9029
:101490000F900F900F90EFCFDF91CF9108950E94A2
:1014A000280A2FEF89E698E1215080409040E1F72B
:1014B00000C0000084E690E00E94CF098093B6024D
:1014C0009093B7029F938F9385EB91E09F938F93B7
:1014D0000E947A070E94370A0F900F900F900F908A
:1014E0008091B6029091B70208950E94DE17909302
:1014F0001501809314010E94D21D80E091E00E94AA
:10150000D9170E94190A0E94200A8111FCCF8DE38D
:1015100092E00E94E1062FEF85EB95E32150804099
:101520009040E1F700C0000089E392E00E944F0A7A
:10153000EFEFFBE42DE1E150F0402040E1F700C087
:1015400000000E94370A85E392E00E944F0AFC01E6
:101550008081863721F081E392E00C944F0A089550
:1015600088E192E00E94E10682E192E00E944F0A47
:101570000E94060A0E94D21D8091140190911501CB
:101580000C94D9170C94580F8F929F92AF92BF92E0
:10159000CF92DF92EF92FF920F931F93CF93DF933F
:1015A00092E0B92E03E614E029E6E22E24E0F22EC2
:1015B000AA24A39433E0932E41E5C42E44E0D42E14
:1015C0000E94CD09EC01019609F441C08091D3023B
:1015D0008130F9F028F0823009F1833021F134C0F4
:1015E000CE3FD10519F4A092D302EACFC038D1057D
:1015F00028F4DF93CF93FF92EF9204C0DF93CF9351
:101600001F930F930E947A070F900F900F900F90E7
:10161000D7CF2297C9F4B092D302D2CF2197A1F4A9
:101620009092D302CDCF8091810380FF0AC0DF93D7
:10163000CF93DF92CF920E947A070F900F900F9076
:101640000F908C2F0E94250A1092D302B9CF80915F
:10165000D502811121C08091D40281111DC00E9448
:101660001C0A81110AC00E94DE178A50914029F09D
:101670000E94D21D8AE091E00DC00E941C0A8823BE
:1016800059F00E94DE178651914031F00E94D21D20
:1016900086E191E00E94D9178091D1029091D20207
:1016A0000E942125893E23E0920708F461C028EEBC
:1016B00033E0B9010E94AE2D629FC001639F900D7F
:1016C000729F900D11242091D1023091D202820F8D
:1016D000931F9093D2028093D1020E94F60F833021
:1016E00011F481E001C080E00E94470F0E9415259F
:1016F00028EE33E040E050E00E94D62D49015A0127
:101700008CE3C82ED12CE12CF12CCA01B901A70120
:1017100096010E94D62D672B682B692B49F50E94F4
:10172000BF0F2091810320FF23C09F938F931F92AF
:101730001F92C501B40120E13EE040E050E00E946C
:10174000D62DC22FA70196010E94D62D3F932F932D
:101750001F92CF938CE394E09F938F930E947A071C
:101760008DB79EB70A960FB6F8949EBF0FBE8DBF79
:101770000E941C0A811107C00E94200A882319F0C8
:101780006E9A769802C06E9A769ADF91CF911F91E9
:101790000F91FF90EF90DF90CF90BF90AF909F9010
:1017A0008F9008958F929F92AF92BF92CF92DF92C7
:1017B000EF92FF921F93CF93DF9300D000D0CDB76D
:1017C000DEB7833109F48CC008F05BC08B3009F4BC
:1017D00066C08C3009F48FC0853009F0FBC10E94CF
:1017E000152528EE33E040E050E00E94D62D490157
:1017F0005A010E94BF0F9F938F938BE892E09F93B3
:101800008F930E947A07C501B40120E13EE040E0D9
:1018100050E00E94D62D5F934F933F932F9325E87E
:1018200032E03F932F9369837A838B839C830E945A
:101830007A078CE3C82ED12CE12CF12C69817A81B6
:101840008B819C81A70196010E94D62D5F934F93B7
:101850003F932F938FE792E09F938F930E947A0795
:10186000C501B401A70196010E94D62D9F938F93C5
:101870007F936F9389E792E09F938F930E947A07FB
:1018800040C1883361F020F4883109F440C1A2C11D
:10189000873409F46DC18C3409F456C19BC188E1C9
:1018A00094E00E94E10683E094E00E94E10689EE64
:1018B00093E00E94E10682EC93E00E94E10687EA51
:1018C00093E00E94E10685E993E00E94E106109111
:1018D000D50211117DC185E793E00E94E1067EC12A
:1018E0000E94750A8DE592E00E944F0A87E592E01A
:1018F0000E944F0A6BC18CE593E00E94E1060E94B2
:10190000DE178A50914019F08FE291E002C089E21F
:1019100091E09F938F938EE493E09F938F930E9427
:101920007A078091D4021F928F938FE393E09F9365
:101930008F930E947A070E941C0A0FB6F894DEBFAC
:101940000FBECDBF811107C00E94200A811106C0C1
:1019500088E391E005C084E391E002C08BE391E06D
:101960009F938F9385E393E09F938F930E947A07D1
:101970000E94010A1F928F938AE193E09F938F93B5
:101980000E947A078091D5021F928F9389E093E09D
:101990009F938F930E947A07809196030FB6F894D5
:1019A000DEBF0FBECDBF8823B9F080919603813092
:1019B000B1F0809196038230A9F080919603833034
:1019C000A1F080919603843099F080919603853040
:1019D00091F080E791E011C088E491E00EC080E4CE
:1019E00091E00BC083E591E008C08BE591E005C074
:1019F00085E691E002C082E791E09F938F938AEFA2
:101A000092E09F938F930E947A0780EF92E09F93DA
:101A10008F930E947A070E94F60F0F900F900F90FD
:101A20000F900F900F90813059F038F0823059F0BC
:101A3000833061F48AED92E00BC08BEE92E008C037
:101A400085EE92E005C08EED92E002C088ED92E056
:101A50009F938F930E947A070F900F9086ED92E0EC
:101A60009F938F930E947A07809194031F928F9384
:101A70008DEB92E09F938F930E947A078091D9001B
:101A800081701F928F9383EB92E09F938F930E94BC
:101A90007A070E94152528EE33E040E050E00E94CE
:101AA000D62D69017A019CE3892E912CA12CB12CB1
:101AB000CA01B901A50194010E94D62D7F936F93AD
:101AC000C701B60120E13EE040E050E00E94D62D83
:101AD000122FA50194010E94D62D3F932F931F92A0
:101AE0001F93C701B60120E831E541E050E00E94B4
:101AF000D62D3F932F9386E992E09F938F930E9478
:101B00007A070FB6F894DEBF0FBECDBF61C08091DB
:101B1000D502811162C01091D402112339F08EE6F2
:101B200092E00E94E1061092D40258C084E692E04E
:101B30000E94E10681E08093D4020E94D21D86E1DA
:101B400091E00E94D91744C00E94010A182F8823EF
:101B500041F00E94750A81E0809391038093D50241
:101B60003DC00E94B00A109291031092D50230C07D
:101B70008091D502811102C00E94750A8BE092E02B
:101B80000E944F0A80E092E00E944F0A8CEE91E0A2
:101B90000E944F0A85EE91E00E944F0A8BED91E082
:101BA0000E944F0A84ED91E00E944F0A8AEC91E076
:101BB0000E944F0A80EC91E00E944F0A8AEB91E06C
:101BC0000E944F0A8091D502811102C00E94B00A82
:101BD00011E004C01091D50201C010E0812F0F90D8
:101BE0000F900F900F90DF91CF911F91FF90EF908A
:101BF000DF90CF90BF90AF909F908F900895CF933C
:101C0000C82F0E94CB23827291E009F490E04C2F00
:101C100050E0FA013497E934F10508F0D0C0EA5AEF
:101C2000FF4F0C94F82D8BE12DC19111CCC081E6B2
:101C300029C19111CAC082E625C19111C8C083E6AD
:101C400021C19111C6C084E61DC19111C4C085E6B1
:101C500019C19111C2C086E615C19111C0C087E6B5
:101C600011C19111BEC088E60DC19111BCC089E6B9
:101C700009C19111BAC08AE605C19111B8C08BE6BD
:101C800001C19111B6C08CE6FDC09111B4C08DE6C2
:101C9000F9C09111B2C08EE6F5C09111B0C08FE6C7
:101CA000F1C09111AEC080E7EDC09111ACC081E7E9
:101CB000E9C09111AAC082E7E5C09111A8C083E7ED
:101CC000E1C09111A6C084E7DDC09111A4C085E7F1
:101CD000D9C09111A2C086E7D5C09111A0C087E7F5
:101CE000D1C091119EC088E7CDC091119CC089E7F9
:101CF000C9C091119AC08AE7C5C0911198C081E30B
:101D0000C1C0911196C082E3BDC0911194C083E31C
:101D1000B9C0911192C084E3B5C0911190C085E320
:101D2000B1C091118EC086E3ADC091118CC087E324
:101D3000A9C091118AC088E3A5C0911188C089E328
:101D4000A1C0911186C080E39DC088E09BC089E05E
:101D500099C080E297C091117EC08DE293C091112D
:101D60007CC08DE38FC091117AC08BE58BC091113F
:101D700078C08DE587C0992309F475C08CE782C0CF
:101D8000992309F472C08CE77DC0911170C08BE378
:101D900079C091116EC087E275C091116CC080E668
:101DA00071C091116AC08CE26DC0911168C08EE261
:101DB00069C0911166C08FE265C080E063C080E2B7
:101DC00061C08AE05FC081E45DC082E45BC083E4FF
:101DD00059C084E457C085E455C086E453C087E405
:101DE00051C088E44FC089E44DC08AE44BC08BE405
:101DF00049C08CE447C08DE445C08EE443C08FE405
:101E000041C080E53FC081E53DC082E53BC083E540
:101E100039C084E537C085E535C086E533C087E540
:101E200031C088E52FC089E52DC08AE52BC081E24D
:101E300029C080E427C083E225C084E223C085E274
:101E400021C08EE51FC086E21DC08AE21BC088E269
:101E500019C089E217C08FE515C08BE213C08BE76C
:101E600011C08DE70FC08CE50DC08CE50BC08AE377
:101E700009C082E207C08EE705C08CE303C08EE391
:101E800001C08FE30E94FF0981E0CF910895833064
:101E900019F4859A7D9A0895813011F4859A06C0C7
:101EA000823019F4859A8D9A089585988D980895B1
:101EB00081E00E94470F2FEF81EE94E02150804097
:101EC0009040E1F700C0000082E00E94470F2FEF32
:101ED00081EE94E0215080409040E1F700C0000086
:101EE00081E00E94470F2FEF81EE94E02150804067
:101EF0009040E1F700C0000082E00E94470F2FEF02
:101F000081EE94E0215080409040E1F700C0000055
:101F100080E00E94470F80EC80937C0087E08093F4
:101F20007A0081E980937E0081E080937F008BE3DB
:101F300080937D00849A8C9808958091D90080FFC9
:101F40001CC090B331B385988D9AEFE9FFE03197CB
:101F5000F1F700C000008FB185FB882780F920B31E
:101F600090722F7D292B20BB91B3232F20729F7D50
:101F7000922B91BB91E08927089580E00895CF933B
:101F8000DF9300D0CDB7DEB7849A8C9A80917A0027
:101F9000806880937A008FE99FE00197F1F700C095
:101FA000000080917A00806480937A0080917A00AA
:101FB00086FDFCCF80917800909179009A83898387
:101FC00080917A008F7780937A00849A8C98298107
:101FD0003A8145E0429FC001439F900D11248055F6
:101FE00091090F900F90DF91CF9108958091D900C2
:101FF00080FD0C949D0F0E94BF0F8C3A2DE092073C
:1020000020F481E08093D60205C085379E4010F011
:102010001092D6028091D602811102C082E008950A
:1020200083E00895CF93C82F0E949E068C2F0E94B4
:102030009F1080E0CF91089584B7877F84BF0FB64B
:10204000F894A89580916000886180936000109258
:1020500060000FBE90E080E80FB6F89480936100B6
:10206000909361000FBE0E94F7140E945415809156
:10207000E20084608093E20082E190E10E946724A4
:10208000509A589A5198599A78948FEF9091960354
:102090008150943041F0EFE7FEE33197F1F700C053
:1020A00000008111F3CF8CE894E00E94E1060E94C9
:1020B000090A0E94C20A80E894E00E94E1060E9498
:1020C0009F180E941C0A811103C08AE091E002C09F
:1020D00086E191E00E94D91780E794E00E94E10632
:1020E0000E941C0A882319F1809196038530F9F427
:1020F0008CE694E00E94E1060E949D080E949624CE
:102100000E9496240E9496240E9496240E9496245F
:102110000E9496240E94962480919403882301F3C0
:102120000E94BF248823E1F20E944C13D9CF0E9461
:10213000A3180E94C40AD4CF8091E30208959FB7E8
:10214000F8941092DA029FBF90919603943009F0B0
:1021500057C09091E9009F703091EC00232F2170BF
:1021600030FD20E8922B24E02093E9002091EB0041
:1021700020FF43C02091EE0027FF3FC02091D702EF
:10218000222321F02091E80025FF37C01092D702CA
:1021900026E03091E80035FD15C0309196033430CB
:1021A00061F53091EB0035FD28C0215021F481E02C
:1021B0008093D70222C0EFE9FFE03197F1F700C02A
:1021C0000000E7CF8093F1008091E80085FD0AC010
:1021D0008091E80080FFFCCF8091E8008E778093AB
:1021E000E80006C08FB7F89421E02093DA028FBF91
:1021F0009F709093E90080E008959F709093E900AC
:102200008FEF0895CF93DF9300D01F92CDB7DEB745
:102210009C0180919603843019F593E099833B8368
:102220002A839093E9008FEF9091E800815095FD0B
:1022300006C095ED9A95F1F700008111F5CF8091D8
:10224000E80085FF0DC040E050E063E070E0CE01A3
:1022500001960E9462138091E8008E778093E800D7
:102260000F900F900F90DF91CF910895CF93DF9350
:1022700000D01F92CDB7DEB720919603243021F510
:1022800022E029839B838A8383E08093E9008FEF98
:102290009091E800815095FD06C095ED9A95F1F773
:1022A00000008111F5CF8091E80085FF0DC040E06E
:1022B00050E063E070E0CE0101960E9462138091CD
:1022C000E8008E778093E8000F900F900F90DF91D9
:1022D000CF910895209196032430F1F422E02093C9
:1022E000E9002FEF3091E800215035FD06C035EDB3
:1022F0003A95F1F700002111F5CF2091E80025FF74
:102300000BC040E050E065E070E00E9462138091F5
:10231000E8008E778093E8000895CF93DF932091B3
:102320009603243039F521E02093E9002FEF309116
:10233000E800215035FD06C035ED3A95F1F7000073
:102340002111F5CF2091E80025FF14C0EC0140E0F9
:1023500050E068E070E00E9462138091E8008E77A0
:102360008093E80088E0FE01ABEDB2E001900D92B1
:102370008A95E1F7DF91CF9108958BE994E00E946F
:10238000E10680919503811109C00E94F7140E9413
:1023900054158091E20084608093E200089587E9FB
:1023A00094E00E94E106109295030895089520910B
:1023B000D8022F5F822F62E30E94A22D992319F089
:1023C0002093D80208951092D8028091DA028823CF
:1023D00071F180919603843041F58091E9008F700E
:1023E0002091EC00922F917020FD90E8892B94E0D1
:1023F0009093E9009091EB0090FF14C09091EE0053
:1024000097FF10C09091E80095FF03C01092F10073
:10241000F9CF9091E80090FF05C09091E8009E7779
:102420009093E8008F708093E9001092DA0208958B
:1024300042E061EC81E00E94711442E061EC82E0D4
:102440000E94711442E061EC83E00E94711442E248
:1024500061EC84E00C94711480919803833009F44A
:1024600053C030F4813071F0823009F48CC008958B
:102470008A3009F478C08B3009F45EC0893009F0E5
:102480009AC020C080919703813A09F094C080914E
:10249000E800877F8093E80080919B0390919C03E4
:1024A000892B21F468E08BED92E003C060E080E0CE
:1024B00090E070E00E94AD138091E8008B778093EC
:1024C000E800089580919703813209F074C08091EB
:1024D0009B0390919C03892B09F06DC08091E800CB
:1024E000877F8093E8008091E80082FD05C080919D
:1024F00096038111F8CF5FC08091F1008093E302D1
:102500008091E8008B7753C080919703813A09F05E
:1025100052C080919B0390919C03892B09F04BC082
:102520008091E800877F8093E8008091E80080FF39
:10253000FCCF8091200136C0809197038132D9F57C
:1025400080919B0390919C03892BA9F58091E800D1
:10255000877F8093E8000E94A6148091990380935E
:1025600020010C94D21D80919703813221F5809136
:10257000E800877F8093E8000E94A61480919A0368
:102580008093E402089580919703813AA1F48091A9
:10259000E800877F8093E8008091E80080FFFCCF0F
:1025A0008091E4028093F1008091E8008E7780931F
:1025B000E8000C94A61408958091E3028093D90258
:1025C0001092E30280E00E949F080E9470190C9410
:1025D000D21D0C94DC120E94D3248091D9028093E6
:1025E000E30208950C94EB12292F33272330310591
:1025F000C9F064F42130310581F02230310509F051
:1026000043C084E790E027EC34E042C0213231053A
:10261000F1F02232310541F137C082E190E02BE345
:1026200035E036C099278130910541F0823091051F
:1026300041F0892B49F5E3ECF4E005C0E3EBF4E06D
:1026400002C0EFE9F4E0849190E09F0121C0643082
:10265000D8F4E62FF0E0EE0FFF1FE857FE4F208181
:10266000318189E090E014C0643070F470E0FB01C7
:10267000EE0FFF1FE058FE4F20813181FB01E4582F
:10268000FE4F808190E004C080E090E020E030E0E8
:10269000FA0131832083089580E189BD82E189BDFB
:1026A00009B400FEFDCF8091D8008F7D8093D800C3
:1026B0008091E00082608093E0008091E00081FDE5
:1026C000FCCF0895CF92DF92EF92FF920F931F936A
:1026D000CF93DF93EC018B016A010E94C514811135
:1026E00033C0C114D10439F0F60180819181081BF7
:1026F000190BC80FD91FE12CF12C0115110519F187
:102700008091E80085FD16C08091E8008E77809367
:10271000E800C114D10449F0F60180819181E80EEE
:10272000F91EF182E08285E00FC00E94C514882363
:1027300021F30AC089918093F10001501109FFEF44
:10274000EF1AFF0ADACF80E0DF91CF911F910F914E
:10275000FF90EF90DF90CF90089520919D033091EE
:102760009E032617370748F06115710539F420914B
:10277000E8002E772093E80001C0B90140E0611520
:102780007105A9F120919603222309F443C0253055
:1027900009F442C02091E80023FD40C02091E800E8
:1027A00022FD32C02091E80020FFE9CF4091F300E4
:1027B0002091F20030E0342BFC01CF01611571054E
:1027C00059F02830310540F481918093F100615037
:1027D00071092F5F3F4FF1CF41E02830310509F0FB
:1027E00040E02091E8002E772093E800C8CF411107
:1027F000C9CF0AC080919603882361F0853061F0CB
:102800008091E80083FD0AC08091E80082FFF2CF4A
:1028100080E0089582E0089583E0089581E00895BE
:1028200020919D0330919E032617370748F06115CC
:10283000710539F42091E8002E772093E80001C05B
:10284000B901FC0120E06115710591F180919603B9
:10285000882309F440C0853009F43FC08091E80026
:1028600083FD3DC08091E80082FD2FC08091E8008B
:1028700080FFE9CF2091F3008091F20090E0922B4D
:102880006115710559F08830910540F42491209329
:10289000F1003196615071090196F2CF21E008975D
:1028A00009F020E08091E8008E778093E800CBCF9C
:1028B0002111CCCF0AC080919603882361F0853026
:1028C00061F08091E80083FD0AC08091E80082FFFA
:1028D000F2CF80E0089582E0089583E0089581E0DA
:1028E0000895982F973058F59093E900981739F08C
:1028F0007091EC002091ED005091F00003C0242F66
:10290000762F50E021FF19C03091EB003E7F3093CD
:10291000EB003091ED003D7F3093ED003091EB0006
:1029200031603093EB007093EC002093ED005093F6
:10293000F0002091EE0027FF07C09F5FD3CF8F707C
:102940008093E90081E0089580E0089580919703E5
:1029500087FF11C08091E80082FD05C08091960339
:102960008111F8CF11C08091E8008B770BC0809166
:102970009603882349F08091E80080FFF8CF80918A
:10298000E8008E778093E80008952091E40030916C
:10299000E50095E64091EC00842F817040FF22C055
:1029A0008091E80080FD1CC080919603882391F0FF
:1029B000853091F08091EB0085FD10C04091E400DE
:1029C0005091E5004217530729F39A01915011F7EE
:1029D00084E0089582E0089583E0089581E00895F9
:1029E00080E008954091E80042FFDECF08950E9404
:1029F00065150E946D15E0EEF0E0808181608083B6
:102A0000E8EDF0E080818F77808319BCA7EDB0E01E
:102A10008C918E7F8C9380818F7E80831092950322
:102A200008950F931F93CF93DF930E9465150E9423
:102A30006D15C8EDD0E088818F77888388818068A4
:102A4000888388818F7D888319BC109296031092A9
:102A50009203109294031092930300EE10E0F80199
:102A600080818B7F808388818160888342E060E001
:102A700080E00E947114E1EEF0E080818E7F80831F
:102A8000E2EEF0E0808181608083808188608083D5
:102A9000F80180818E7F8083888180618883DF91C7
:102AA000CF911F910F910895E8EDF0E080818F7E26
:102AB0008083E7EDF0E080818160808384E082BFE5
:102AC00081E0809395030C941115E8EDF0E080818E
:102AD0008E7F80831092E20008951092DA001092A7
:102AE000E10008951F920F920FB60F9211242F93B9
:102AF0003F934F935F936F937F938F939F93AF9386
:102B0000BF93EF93FF938091E10082FF0BC0809110
:102B1000E20082FF07C08091E1008B7F8093E1009B
:102B20000E94D7118091DA0080FF1FC08091D800E9
:102B300080FF1BC08091DA008E7F8093DA00809145
:102B4000D90080FF0DC080E189BD82E189BD09B453
:102B500000FEFDCF81E0809396030E94BD1105C069
:102B600019BC109296030E94CF118091E10080FF62
:102B700019C08091E20080FF15C08091E2008E7F35
:102B80008093E2008091E20080618093E200809176
:102B9000D80080628093D80019BC85E080939603AA
:102BA0000E94E9128091E10084FF30C08091E20030
:102BB00084FF2CC080E189BD82E189BD09B400FE9B
:102BC000FDCF8091D8008F7D8093D8008091E10067
:102BD0008F7E8093E1008091E2008F7E8093E200FF
:102BE0008091E20081608093E200809192038823CB
:102BF00011F084E007C08091E30087FD02C081E00E
:102C000001C083E0809396030E94F2128091E1005C
:102C100083FF29C08091E20083FF25C08091E100FD
:102C2000877F8093E10082E0809396031092920365
:102C30008091E1008E7F8093E1008091E2008E7FA1
:102C40008093E2008091E20080618093E20042E0A4
:102C500060E080E00E9471148091F00088608093B1
:102C6000F0000E94D611FF91EF91BF91AF919F911B
:102C70008F917F916F915F914F913F912F910F9025
:102C80000FBE0F901F9018951F920F920FB60F92C4
:102C900011242F933F934F935F936F937F938F9361
:102CA0009F93AF93BF93CF93DF93EF93FF93C09125
:102CB000E900CF708091EC00D82FD17080FDD0E872
:102CC0001092E9008091F000877F8093F000789463
:102CD0000E9488161092E9008091F000886080932D
:102CE000F000CD2BCF70C093E900FF91EF91DF9101
:102CF000CF91BF91AF919F918F917F916F915F9194
:102D00004F913F912F910F900FBE0F901F901895EC
:102D10001F93CF93DF93CDB7DEB7AA970FB6F89482
:102D2000DEBF0FBECDBFE7E9F3E088E08E0F9091E4
:102D3000F10091938E13FBCF0E942C128091E8003A
:102D400083FF1FC18091970390919803492F50E012
:102D50004A30510508F015C1FA01E156FF4F0C94B5
:102D6000F82D803881F0823809F00BC180919B03E7
:102D70008F708093E9008091EB0085FB882780F9B4
:102D80001092E90006C080919303909194039111F1
:102D900082609091E800977F9093E8008093F10023
:102DA0001092F100C8C0282F2D7F09F0EAC08823B7
:102DB00019F0823061F0E5C080919903813009F00B
:102DC000E0C0933009F080E0809394032BC08091A1
:102DD0009903811127C080919B038F7009F4D1C0A2
:102DE0008093E9002091EB0020FF1CC0933021F478
:102DF0008091EB00806214C09091EB009061909301
:102E0000EB0021E030E0A90102C0440F551F8A9574
:102E1000E2F74093EA001092EA008091EB008860AC
:102E20008093EB001092E9008091E800877F86C0D4
:102E30008111A7C0109199031F778091E3008078DA
:102E4000812B8093E3008091E800877F8093E800E6
:102E50000E94A6148091E80080FFFCCF8091E300DF
:102E600080688093E300111102C082E001C083E01A
:102E70008093960386C08058823008F082C080918B
:102E8000990390919A038C3D53E0950779F583E07F
:102E90008A838AE289834FB7F894DE01139620E093
:102EA0003EE051E2E32FF0E050935700E49120FF21
:102EB00003C0E295EF703F5FEF708E2F90E0EA3035
:102EC00010F0C79601C0C0968D939D932F5F24315B
:102ED00049F74FBF8091E800877F8093E8006AE25E
:102EE00070E0CE0101960E94AD1314C0AE014F5F99
:102EF0005F4F60919B030E94F412BC01892B09F47F
:102F000040C09091E800977F9093E80089819A8172
:102F10000E9410148091E8008B778093E80031C004
:102F2000803879F58091E800877F8093E800809170
:102F300092038093F1008091E8008E778093E800FF
:102F40000E94A6141EC081111CC09091990392305A
:102F5000C0F48091E800877F8093E800909392030B
:102F60000E94A61480919203811106C08091E30013
:102F700087FD02C081E001C084E0809396030E9437
:102F800018128091E80083FF0AC08091E800877FD3
:102F90008093E8008091EB0080628093EB00AA961A
:102FA0000FB6F894DEBF0FBECDBFDF91CF911F915A
:102FB00008959093EA028093E90208958091E902CE
:102FC0009091EA020895E091E902F091EA023097C7
:102FD00021F00190F081E02D099480E00895EF92B6
:102FE000FF920F931F93CF93DF93E091E902F0914B
:102FF000EA023097B1F18C010280F381E02D09954E
:103000008091810382FF2DC080FF04C088E596E097
:103010000E94E106E80118E082E5E82E86E0F82E3D
:103020008091810380FF0BC088811F928F93FF9254
:10303000EF920E947A070F900F900F900F9011500F
:1030400021961111EDCF8091810380FF0AC080E5A8
:1030500096E0DF91CF911F910F91FF90EF900C942C
:10306000E106DF91CF911F910F91FF90EF900895AE
:10307000E091E902F091EA02309721F00480F581B5
:10308000E02D09940895CF93DF93EC018091E7023E
:103090009091E802C817D90709F1D093E802C093CC
:1030A000E702E091E902F091EA023097B9F0068078
:1030B000F781E02DCE0109958091810382FF0EC03A
:1030C00080FF0CC0DF93CF9382E496E09F938F93B1
:1030D0000E947A070F900F900F900F90DF91CF9181
:1030E0000895CF93DF93EC018091E5029091E60281
:1030F000C817D90709F1D093E602C093E502E09121
:10310000E902F091EA023097B9F00084F185E02DF0
:10311000CE0109958091810382FF0EC080FF0CC013
:10312000DF93CF9382E396E09F938F930E947A0779
:103130000F900F900F900F90DF91CF9108950E9404
:1031400000250C9496075F926F927F928F929F92C8
:10315000AF92BF92CF92DF92EF92FF920F931F93A5
:10316000CF93DF9300D000D01F92CDB7DEB70E947F
:10317000C1078CEEC82E82E0D82E512C882483946F
:10318000912C852D0E949208A82EF601E080E82659
:1031900041F45394FFEFCF1ADF0A88E05812F1CFC1
:1031A00040C08091810381FD0E94711900E010E010
:1031B000F12CB12CC701002E02C0959587950A9479
:1031C000E2F780FF28C009835A823401002E02C032
:1031D000660C771C0A94E2F793012A213B2181E0D7
:1031E000232B09F480E08B830E9409258160782FCE
:1031F0009D838C8349815A816B818D810E94A519A1
:1032000049815A816B817C818D810E948324F601E2
:103210008081682660820F5F1F4F0830110551F6CC
:10322000B8CF8FEF89838A831B820E940925816032
:10323000782F9D838C8349815A816B818D810E9477
:10324000A5190E9482240E94F6271091EB020E9489
:10325000E317181771F10E94E3178093EB02909126
:10326000810392FF0EC090FF0CC01F928F9383E6E4
:1032700096E09F938F930E947A070F900F900F9084
:103280000F908091EB020F900F900F900F900F9086
:10329000DF91CF911F910F91FF90EF90DF90CF9032
:1032A000BF90AF909F908F907F906F905F900C94A5
:1032B00094240F900F900F900F900F90DF91CF916B
:1032C0001F910F91FF90EF90DF90CF90BF90AF9044
:1032D0009F908F907F906F905F9008950C949F08BF
:1032E0000895EF92FF920F931F93CF93DF938CE794
:1032F00096E00E94E106C0E0D0E08EE2E82E81E098
:10330000F82E0EE616E08C2F0E9492080E946C2484
:10331000FF92EF921F928F93DF93CF931F930F93A0
:103320000E947A0721968DB79EB708960FB6F8943B
:103330009EBF0FBE8DBFC830D10529F7DF91CF9159
:103340001F910F91FF90EF900895CF93DF93CDB72A
:10335000DEB72B970FB6F894DEBF0FBECDBF942F0C
:103360004F83252F588769877A878B874A855B85A6
:10337000452B21F02F3F09F59F3FF9F4DE0111960F
:1033800086E0FD0111928A95E9F785E0FE01379606
:1033900001900D928A95E1F749815A816B817C8178
:1033A0008D819E810E94B7202B960FB6F894DEBFC8
:1033B0000FBECDBFDF91CF9108954F8158856985AC
:1033C0007A858B850E948324D9CFCF93882309F4F3
:1033D00065C0C82F8CEF8C0F813A20F080E58C0FF0
:1033E0008E3248F48C2F0E941C2B811157C08C2FD9
:1033F0000E948F230CC080E28C0F883058F4C77075
:1034000081E001C0880FCA95EAF70E94CE23CF91D0
:103410000C9412248BE58C0F833078F4C53A29F094
:10342000C63A31F083E890E005C081E890E002C040
:1034300082E890E0CF910C94431888E58C0F853199
:1034400068F5C83A89F0C93A91F0CA3A99F0CB3A8E
:10345000A1F0CC3AA9F0CD3AB1F0CE3AB9F0CF3ADA
:10346000C1F080E090E017C082EE90E014C089EED9
:1034700090E011C08AEE90E00EC085EB90E00BC0AA
:1034800086EB90E008C083EB90E005C084EB90E011
:1034900002C087EB90E0CF910C947118CF91089502
:1034A000882349F19CEF980F913A20F090E5980F0E
:1034B0009E3218F40E94AC230DC090E2980F983011
:1034C00058F4877091E001C0990F8A95EAF7892F27
:1034D0000E94D4230C9412249BE5980F933020F47F
:1034E00080E090E00C944318885A853120F480E005
:1034F00090E00C9471180895882321F00E94CE2347
:103500000C9412240895882321F00E94D4230C9453
:1035100012240895BF92CF92DF92EF92FF920F9301
:103520001F93CF93DF9300D000D000D0CDB7DEB78C
:1035300025E0FC01DE01119601900D922A95E1F73C
:10354000FC01408151810281638174812581229532
:103550002F706115710509F403C35F3F19F44F3FE4
:1035600009F4FEC26C01862F7D836C83602F782F57
:103570008D812E830E941323182FB92E0E941223AF
:103580000E940222EB2DE295EF70F0E0E755FF4F2D
:103590002E810C94F82D8B2D807F9B2D9F70F92E02
:1035A000882319F0F29490EFF922002349F0FF20CC
:1035B00009F483C28F2D0E94E1230E9412247DC250
:1035C000812F0E94501AFF2009F4CAC28F2D0E9439
:1035D000E72326960FB6F894DEBF0FBECDBFDF916E
:1035E000CF911F910F91FF90EF90DF90CF90BF9000
:1035F0000C9412248B2D807F9B2D9F70F92E80328E
:1036000019F0F29480EFF822112319F0113009F12A
:103610002AC00023B1F08F2D222351F1213041F532
:1036200026960FB6F894DEBF0FBECDBFDF91CF91C7
:103630001F910F91FF90EF90DF90CF90BF900C946F
:10364000F123222319F0213009F48AC20E94FA23BF
:103650002DC00023F1F0263008F082C20E94CB2357
:103660008F2129F023C00023F9F0211116C08F2DDE
:1036700026960FB6F894DEBF0FBECDBFDF91CF9177
:103680001F910F91FF90EF90DF90CF90BF900C941F
:103690007C1A253008F064C209C0F601858180FFDC
:1036A0000CC28F708583E3CF21111CC28F2D83C183
:1036B0002B2D26952695237030E02115310521F01C
:1036C00021303105D1F04CC2002321F0812F9B2DF8
:1036D000937002C080E090E026960FB6F894DEBFAB
:1036E0000FBECDBFDF91CF911F910F91FF90EF9053
:1036F000DF90CF90BF900C944318002321F0812FCE
:103700009B2D937002C080E090E026960FB6F8944F
:10371000DEBF0FBECDBFDF91CF911F910F91FF9004
:10372000EF90DF90CF90BF900C947118812F002301
:1037300019F00E947C2602C00E94E42626960FB64D
:10374000F894DEBF0FBECDBFDF91CF911F910F91D7
:10375000FF90EF90DF90CF90BF900C9469278B2D56
:10376000837009F07BC00111FBC1812F8295869582
:103770008770880F880F912F9F70C92ED12CE12C54
:10378000F12C082E04C0CC0CDD1CEE1CFF1C0A948E
:10379000D2F714FF12C04FE050E060E070E004C0C8
:1037A000440F551F661F771F8A95D2F7CB01BA01C8
:1037B000609570958095909503C060E070E0CB01B6
:1037C0002B2D269526952370422F50E0423051052F
:1037D000D9F04330510569F16C297D298E299F2943
:1037E0004130510551F126960FB6F894DEBF0FBE59
:1037F000CDBFDF91CF911F910F91FF90EF90DF90A0
:10380000CF90BF900C9427226C297D298E299F2967
:1038100026960FB6F894DEBF0FBECDBFDF91CF91D5
:103820001F910F91FF90EF90DF90CF90BF900C947D
:1038300041220E942722C701B60126960FB6F894AE
:10384000DEBF0FBECDBFDF91CF911F910F91FF90D3
:10385000EF90DF90CF90BF900C940D22002319F0D1
:103860008B2D817001C08695882309F479C1812F41
:10387000829586958770880F880F912F9F70C92E2B
:10388000D12CE12CF12C082E04C0CC0CDD1CEE1C3C
:10389000FF1C0A94D2F714FF12C04FE050E060E022
:1038A00070E004C0440F551F661F771F8A95D2F73A
:1038B000CB01BA01609570958095909503C060E04A
:1038C00070E0CB012B2D269526952370422F50E0DA
:1038D00042305105D9F04330510569F16C297D29F9
:1038E0008E299F294130510551F126960FB6F89443
:1038F000DEBF0FBECDBFDF91CF911F910F91FF9023
:10390000EF90DF90CF90BF900C94EE226C297D2930
:103910008E299F2926960FB6F894DEBF0FBECDBF25
:10392000DF91CF911F910F91FF90EF90DF90CF909B
:10393000BF900C9400230E94EE22C701B601269688
:103940000FB6F894DEBF0FBECDBFDF91CF911F91B0
:103950000F91FF90EF90DF90CF90BF900C94DC22FE
:10396000103FD1F128F480E4810F803250F0A0C0E4
:10397000123F09F462C008F44BC0133F09F472C04F
:1039800097C0F12FF071FF2E8B2D8F71002351F016
:103990000E947522812FFF2019F08295807F68CECA
:1039A0008F7066CE0E949622812FFF2019F082959B
:1039B000807F01C08F7026960FB6F894DEBF0FBED1
:1039C000CDBFDF91CF911F910F91FF90EF90DF90CE
:1039D000CF90BF900C94831A0023B1F0253008F0EB
:1039E000BFC08B2D8F7126960FB6F894DEBF0FBE29
:1039F000CDBFDF91CF911F910F91FF90EF90DF909E
:103A0000CF90BF900C94BB22263008F0A9C0E9CF1C
:103A10000023A9F08B2D8F7126960FB6F894DEBF88
:103A20000FBECDBFDF91CF911F910F91FF90EF900F
:103A3000DF90CF90BF900C947522002359F38B2D0B
:103A40008F7126960FB6F894DEBF0FBECDBFDF9103
:103A5000CF911F910F91FF90EF90DF90CF90BF908B
:103A60000C949622002399F08B2D8F7126960FB619
:103A7000F894DEBF0FBECDBFDF91CF911F910F91A4
:103A8000FF90EF90DF90CF90BF900C94602226962D
:103A90000FB6F894DEBF0FBECDBFDF91CF911F915F
:103AA0000F91FF90EF90DF90CF90BF900C945B222E
:103AB0000023A9F0222309F4ADCF812F26960FB65B
:103AC000F894DEBF0FBECDBFDF91CF911F910F9154
:103AD000FF90EF90DF90CF90BF900C94E5192223D8
:103AE00009F4ADCF812F26960FB6F894DEBF0FBE36
:103AF000CDBFDF91CF911F910F91FF90EF90DF909D
:103B0000CF90BF900C94501A4B2D4F70612FC6016F
:103B10000E94F62526960FB6F894DEBF0FBECDBFE5
:103B2000DF91CF911F910F91FF90EF90DF90CF9099
:103B3000BF900C945B214B2D4F70612FC6012696D0
:103B40000FB6F894DEBF0FBECDBFDF91CF911F91AE
:103B50000F91FF90EF90DF90CF90BF900C94F925DC
:103B600026960FB6F894DEBF0FBECDBFDF91CF9182
:103B70001F910F91FF90EF90DF90CF90BF9008952D
:103B80000E94EE230E94BD230E9412240E949B28C3
:103B90000E94692780E090E00E94431880E090E056
:103BA0000C9471180E94DE230C94C01DCF93DF93F8
:103BB00000D000D01F92CDB7DEB7942F4983252FB8
:103BC0005A836B837C838D834C815D81452B39F1D6
:103BD0002F3F11F49F3F19F149815A816B817C81FC
:103BE0008D810E941323292F22952F7030E02C30D5
:103BF000310504F52A3031055CF4225031092230B8
:103C0000310568F4853A80F4843090F4823080F095
:103C1000883E38F4803E60F48450813A48F080E079
:103C200014C0803FE1F704C090E2980F983080F70D
:103C300081E00BC02C30310521F493FB882780F9FB
:103C400004C02F303105C9F3EACF0F900F900F90C9
:103C50000F900F90DF91CF910895CF93DF9300D015
:103C600000D01F92CDB7DEB70F900F900F900F903E
:103C70000F90DF91CF910895CF93DF9300D000D0C4
:103C800000D0CDB7DEB726960FB6F894DEBF0FBED4
:103C9000CDBFDF91CF9108951F93CF93DF93C09154
:103CA000F40216E08091F502C81799F0D0E01C9F4D
:103CB000F0011D9FF00D1124EA50FD4F408151810C
:103CC00062817381848195810E943C1E2196C77018
:103CD000E9CFDF91CF911F91089540912603509134
:103CE0002703609128037091290380912A03909102
:103CF0002B030C943C1E80912B0382958F7009F04E
:103D000054C080912803882309F44FC08091F402A5
:103D1000A091F50260912603709127034091290339
:103D200050912A03B6E08A1709F43FC090E041158C
:103D30005105C1F17F3F11F46F3FA1F1B89FF00130
:103D4000B99FF00D1124EA50FD4F218172132AC052
:103D50002081621327C02281211124C02381348154
:103D60002417350710F421503109241B350B2C3250
:103D70003140C0F420912B032F70206120932B033E
:103D800026E0289FF001299FF00D1124E550FD4FFA
:103D900080818F708061808386E293E00E948A1A1E
:103DA0000C944C1E01968770BECF0895BF92CF929F
:103DB000DF92EF92FF920F931F93CF93DF93CDB7D4
:103DC000DEB761970FB6F894DEBF0FBECDBF7C01A2
:103DD00085E0F701DE011D9601900D928A95E1F7CD
:103DE000D7014C9111965C9111971296DC90129725
:103DF00013960D911C91149730912603609127031F
:103E00008091290390912A03009709F47FC16F3FA5
:103E100019F43F3F09F47AC1B0902803BB2009F49C
:103E2000CAC020912B030817190750F0F801E81BAE
:103E3000F90BCF01CC24C3948C329140D0F009C04F
:103E400080959095800F911FCC24C3948C32914023
:103E500080F0C12C207F09F0CCC0702F198B088B0B
:103E60006D2D89890E942D1E86E293E00E948A1A98
:103E7000B6C0822F807F09F047C0651314C0341389
:103E800012C0D11010C02F70206120932B030E940C
:103E90006D1E86E293E00E948A1A80912B03D7015F
:103EA00015968C932FC00115110519F15F3F11F480
:103EB0004F3FF9F0CD2CD1101CC08091F40220911D
:103EC000F50236E0821709F45CC090E0389FF001FB
:103ED000399FF00D1124EA50FD4F6181561306C041
:103EE0006081461303C06281611103C0019687702F
:103EF000E9CFCD2CDD2009F429C180912B0381600D
:103F000080932B03C12C22C1651308C0341306C053
:103F1000D11004C080912B03D701CCC04D875E87A0
:103F2000DF86702F198B088B6D2D89890E94D61D15
:103F30008823E9F1DD20D9F120912B03822F82958E
:103F40008F7090E0029774F0809126039091270380
:103F500098878F8319861B870A872C87CE0107963F
:103F60000E948A1A86E0F701A6E2B3E001900D9262
:103F70008A95E1F70E947B1E0E946D1ECC24C3949B
:103F8000E5C0702F198B088B60E089890E9413238C
:103F9000292F22952F7030E0223031050CF0CAC055
:103FA0009F7009F0C4C0805E883008F4CFC0C7019C
:103FB0000E948A1AE3CF0817190708F456C0F801BF
:103FC000E81BF90BCF018C32914008F456C0C12C8C
:103FD000702F198B088B6D2D89890E942D1EE6E2AA
:103FE000F3E086E0DF011D928A95E9F70E946D1EDD
:103FF000ADC0651314C0341312C0D11010C080912D
:104000002B03F7018583C7010E948A1A86E0E6E246
:10401000F3E0DF011D928A95E9F7CB2C97C04D871D
:104020005E87DF86702F198B088B6D2D89890E9422
:10403000D61D882309F4BBCFDD2009F4B8CF209129
:104040002B03822F82958F7090E002970CF48ACF19
:1040500080912603909127039A8389831B821D8375
:104060000C832E83CE0101967BCF80959095800F97
:10407000911F8C32914008F0AACFCD2CDD2009F49D
:1040800096CF65132EC034132CC020912B0320FD36
:104090001FC0822F82958F70D9F0D70115962C936F
:1040A00015978F3049F08F5F982F9295907F822FD0
:1040B0008F70892B15968C93C7010E948A1A86E00F
:1040C000F701A6E2B3E001900D928A95E1F78ECF59
:1040D00086E0F701A6E2B3E001900D928A95E1F740
:1040E00035C04D875E87DF86702F198B088B6D2D4D
:1040F00089890E94D61D811135CF80912B03816063
:1041000080932B03C7010E948A1A20C0DD2009F486
:104110004ECF4D875E87DF86702F198B088B6D2DF4
:1041200089890E94D61D882309F441CF1BCF8111B4
:104130003ACF0CC0243031050CF039CF9F7009F410
:1041400032CFF7019581907F09F02DCF8C2D6196AC
:104150000FB6F894DEBF0FBECDBFDF91CF911F9198
:104160000F91FF90EF90DF90CF90BF9008951F9335
:10417000CF93DF93CDB7DEB72C970FB6F894DEBFA1
:104180000FBECDBF4F83588769877A878B879C87FF
:10419000CE0107960E94D61E882369F08F819885EC
:1041A0002A853B85232BF1F19F3F09F063C08F3FA8
:1041B00009F060C037C086E0FE013796DE01119637
:1041C00001900D928A95E1F76F817885EA85FB85EC
:1041D000309741F17F3F11F46F3F21F12091F502BB
:1041E00030E0C9010196877099274091F40250E0B0
:1041F0008417950709F447C069837A83FD83EC83AC
:1042000096E0929FD001939FB00D1124AA50BD4F0C
:10421000FE01319601900D929A95E1F78093F50297
:104220000E944C1E16E08091F4029091F5028917CD
:10423000C1F1189FC00111248A509D4F0E94D61EC3
:10424000882379F1E091F4021E9FF0011124EA50D5
:10425000FD4F4081518162817381848195810E94EB
:104260003C1E8091F40290E001968770992780931C
:10427000F402D9CF4F81588569857A858B859C85D5
:104280000E943C1ECFCF0E94D21D1092F5021092C8
:10429000F402E6E2F3E086E0DF011D928A95E9F799
:1042A000C1CF2C960FB6F894DEBF0FBECDBFDF9105
:1042B000CF911F910895DF92EF92FF920F931F937A
:1042C000CF93DF93FC01892B09F48AC0E12CF12CF8
:1042D000DD24D394EF0121968491853709F461C0E0
:1042E00058F4843708F04EC0843008F06AC081303A
:1042F000D1F0823071F174C0883709F45DC050F498
:10430000863709F455C0873709F06AC08E2D0E94A0
:10431000DB2354C09CE7980F903708F061C08F777B
:104320000E94501A50C08F010E5F1F4FFE018491F2
:1043300090E2980F983050F48770FD2D01C0FF0F68
:104340008A95EAF78F2F0E94E12314C00E94E51995
:1043500013C08F010E5F1F4FFE01C49180E28C0FCE
:10436000883060F4C7708D2D01C0880FCA95EAF7B8
:104370000E94E7230E941224E80125C08C2F0E948E
:10438000501AFACF9F012E5F3F4FFE01C491CC23FC
:1043900069F08FE99FE00197F1F700C00000C1507C
:1043A000F6CF9F012E5F3F4FFE01F490E9010BC055
:1043B0000E94CB23E82E07C00E94DE230E94122415
:1043C00002C00E94E5198F2D882341F0EFE9FFE03C
:1043D0003197F1F700C000008150F6CFFE017ACF8F
:1043E000DF91CF911F910F91FF90EF90DF90089593
:1043F00060936C0370936D0380936E0390936F03CF
:104400000C949324089560937003709371038093C8
:104410007203909373030C9492240F931F93009153
:104420007003109171032091720330917303602B1C
:10443000712B822B932B6093700370937103809385
:104440007203909373031F910F910C9492240F9316
:104450001F930091700310917103209172033091AA
:1044600073036023712382239323609370037093FB
:10447000710380937203909373031F910F910C94B7
:1044800092240F931F930091700310917103209158
:1044900072033091730360277127822793276093FB
:1044A00070037093710380937203909373031F9151
:1044B0000F910C94922460E070E0CB010C94F821F1
:1044C0000F931F9341E050E060E070E08A019B0190
:1044D00004C0000F111F221F331F8A95D2F7C90194
:1044E000B8011F910F910C94F8210F931F9341E095
:1044F00050E060E070E004C0440F551F661F771F56
:104500008A95D2F780916C0390916D03A0916E0310
:10451000B0916F038A019B01082B192B2A2B3B2B8F
:10452000C901B8011F910F910C94F8210F931F93AB
:1045300041E050E060E070E004C0440F551F661F8A
:10454000771F8A95D2F74095509560957095809128
:104550006C0390916D03A0916E03B0916F038A017B
:104560009B01082319232A233B23C901B8011F916A
:104570000F910C94F8210F931F9341E050E060E0FD
:1045800070E004C0440F551F661F771F8A95D2F74D
:1045900080916C0390916D03A0916E03B0916F03B5
:1045A0008A019B01082719272A273B27C901B8013F
:1045B0001F910F910C94F8210F931F9300916C039E
:1045C00010916D0320916E0330916F03602B712B5E
:1045D000822B932B1F910F910C94F8210F931F9313
:1045E00000916C0310916D0320916E0330916F0365
:1045F00060237123822393231F910F910C94F82140
:104600000F931F9300916C0310916D0320916E0323
:1046100030916F0360277127822793271F910F9195
:104620000C94F82108958F929F92AF92BF92DF92DF
:10463000EF92FF920F931F93CF93DF9300D000D0A0
:104640001F92CDB7DEB76B837C838D838A018C810B
:104650009D81892B21F01F3F29F44F3F19F480E001
:1046600090E04CC08B818823C9F1809070039090BA
:104670007103A0907203B090730380916C039091CA
:104680006D03A0916E03B0916F03882A992AAA2A1C
:10469000BB2A8FE1E82EF12CD501C4010E2C04C0F9
:1046A000B695A795979587950A94D2F780FF07C08E
:1046B000DE2CB8018E2D0E94CC25019729F481E0D3
:1046C000E81AF10848F7D12C88E0189FF00111246E
:1046D000E00FF11DE45DFC4FD08209C088E0189F17
:1046E000F0011124E00FF11DE45DFC4FD08009833F
:1046F0001A8369817A818D2D0E94CC250F900F90AD
:104700000F900F900F90DF91CF911F910F91FF901D
:10471000EF90DF90BF90AF909F908F900895209181
:10472000210130912201F90132969FEF40E0519131
:10473000581789F09F3F19F4511101C0942F4F5F12
:104740004630A9F79F3F39F0F901E90FF11D97FDB8
:10475000FA958283089508952091210130912201D4
:10476000F9013296285F3F4F9081981301C0108263
:104770003196E217F307C1F7089581E090E0E091E8
:104780002101F0912201E80FF91F10820196883073
:104790009105A9F708958091800308959091800371
:1047A000892B8093800308958095909180038923BD
:1047B000809380030895809380030895109280036E
:1047C000089590917F03892B80937F0308958095AE
:1047D00090917F03892380937F03089510927F0334
:1047E0000895809376030E94092590937503809322
:1047F0007403089510927603109275031092740357
:1048000008958091210190912201FC0131969C0133
:10481000285F3F4F80E0919191118F5FE217F3077E
:10482000D1F70895E0912101F09122018091800358
:104830008083E0912101F0912201908180917F039A
:10484000892B8083809176038823D9F10E940925E2
:1048500020917403309175038217930748F00E94EA
:1048600009252091740330917503821B930B0AC0B4
:104870000E9409252091740330917503209530958D
:10488000820F931F8C32914070F08091810380FFE2
:1048900008C08AE896E09F938F930E947A070F9052
:1048A0000F900E94FA23E0912101F0912201908162
:1048B00080917603892B80830E94012481110E94BC
:1048C000FA2380912101909122010C94EF1790938B
:1048D0009B0180939A0108958295982F9C7C392F93
:1048E00036953695282F237344E0249FC001112468
:1048F000932F982B292F2A7A2695892F8575880F33
:10490000822B08950895CF93DF9300D000D01F929B
:10491000CDB7DEB70F900F900F900F900F90DF91F3
:10492000CF910895089508950C946E19809196037F
:10493000843021F11092820320E488E190E00FB6E8
:10494000F894A895809360000FBE2093600083B711
:10495000817F846083BF83B7816083BF78948895AB
:1049600083B78E7F83BF0FB6F894A89580916000BF
:10497000886180936000109260000FBE0895CF930D
:104980000E949B080E94C1070E949D08C0E08C2FD6
:104990000E949208811104C0CF5FC830C1F701C0E6
:1049A00081E0CF9108950E9470190C94D21D1F923E
:1049B0000F920FB60F9211248F939F93AF93BF93D3
:1049C00080918203811113C08091830390918403AD
:1049D000A0918503B09186034196A11DB11D8093DE
:1049E000830390938403A0938503B0938603BF91C0
:1049F000AF919F918F910F900FBE0F901F901895C0
:104A000082E084BD93E095BD9AEF97BD80936E00E0
:104A100008952FB7F8948091830390918403A09117
:104A20008503B09186032FBF08952FB7F894609146
:104A300083037091840380918503909186032FBF37
:104A40000895CF92DF92EF92FF920F931F932FB7AB
:104A5000F894409183035091840360918503709191
:104A600086032FBF6A017B01EE24FF248C0120E026
:104A700030E0C016D106E206F30610F441505109A9
:104A80009A01281B390BC9011F910F91FF90EF90DC
:104A9000DF90CF900895CF92DF92EF92FF920F9325
:104AA0001F932FB7F894C0908303D0908403E090B5
:104AB0008503F09086032FBF97018601061B170B15
:104AC000280B390BC616D706E806F90618F0C901F7
:104AD000B80106C0C901B801615071098109910985
:104AE0001F910F91FF90EF90DF90CF9008951F924C
:104AF0000F920FB60F9211248F939F93AF93BF9392
:104B00008091830390918403A0918503B0918603E3
:104B10000196A11DB11D8093830390938403A093FC
:104B20008503B0938603BF91AF919F918F910F90B2
:104B30000FBE0F901F9018950E94F714F8942FEF56
:104B400087EA91E6215080409040E1F700C00000E4
:104B500087E090EBDC0180939F039093A003A093E8
:104B6000A103B093A2039CE088E10FB6F894A89546
:104B7000809360000FBE90936000FFCF28E0929F6B
:104B8000F0011124E80FF11DEE58FE4F9491892F8A
:104B90008F7092959F700895CF93C82FCB010E947C
:104BA000BE25282F30E080E1989FA0011124422BE0
:104BB000532B4038510519F480E090E015C09770F0
:104BC000E92FF0E088E0C89FE00DF11D112484E09A
:104BD000EE0FFF1F8A95E1F7E20FF31FEE0FFF1FA5
:104BE000E050F84985919491CF91089580E090E04C
:104BF000089508958091890380FF0BC0609126017C
:104C000085E0689FB0011124759567957595679546
:104C10002BC081FF09C06091260185E0689FB0012B
:104C200011247595679520C082FF07C06091260109
:104C300085E0689FB001112417C090918A039923E1
:104C4000D1F060912501961788F72091260185E023
:104C5000289F90011124929FA001939F500D112431
:104C600070E0CA010E94C22D6038710540F46115E0
:104C7000710539F002C065E070E0862F08958FE776
:104C8000089581E008958091890380FF08C06091B4
:104C9000240170E0759567957595679521C081FF32
:104CA00006C06091240170E07595679519C082FF78
:104CB00004C06091240170E010C090918A03992390
:104CC000C1F0609123019617A0F780912401899F7C
:104CD000C001112470E00E94C22D6038710528F4D3
:104CE0006115710521F0862F08958FE7089581E001
:104CF000089561E070E0F4CF803F21F40E94FA252E
:104D0000819504C0813F29F40E94FA2580938D0388
:104D10000895823F21F40E94FA25819504C0833FC3
:104D200029F40E94FA2580938C030895893F19F491
:104D30000E94432605C08A3F31F40E944326819594
:104D400080938E0308958B3F21F40E944326819522
:104D500004C08C3F29F40E94432680938F0308955A
:104D6000843F21F480918B03816017C0853F21F43B
:104D700080918B03826011C0863F21F480918B0368
:104D800084600BC0873F21F480918B03886005C04D
:104D9000883F31F480918B03806180938B03089569
:104DA0008D3F21F48091890381600BC08E3F21F4F7
:104DB00080918903826005C08F3F29F48091890327
:104DC0008460809389030895803F39F480918D0336
:104DD00087FF6CC010928D0369C0813F29F48091D8
:104DE0008D031816BCF362C090918C03823F29F4A6
:104DF00097FF5CC010928C0359C0833F19F41916B9
:104E0000CCF354C0893F41F480918E0318160CF006
:104E10004DC010928E034AC08A3F29F480918E03C0
:104E200087FF44C0F6CF8B3F39F480918F0387FF13
:104E30003DC010928F033AC08C3F29F480918F03BC
:104E40001816BCF333C0843F21F480918B038E7F0E
:104E500017C0853F21F480918B038D7F11C0863F61
:104E600021F480918B038B7F0BC0873F21F48091CD
:104E70008B03877F05C0883F31F480918B038F7E41
:104E800080938B0313C08D3F21F4809189038E7F23
:104E90000BC08E3F21F4809189038D7F05C08F3F29
:104EA00029F4809189038B7F8093890380918C03FF
:104EB00081110EC080918D0381110AC080918E03F3
:104EC000811106C080918F03811102C010928A0364
:104ED00008958091810383FF7EC083EC96E00E9459
:104EE000E10680918B031F928F938EEB96E09F9348
:104EF0008F930E947A078CEB96E00E94E1068091E6
:104F00008C03282F082E000C330B3F938F9389EBD3
:104F100096E09F938F930E947A0787EB96E00E941A
:104F2000E10680918D03282F082E000C330B3F9350
:104F30008F9384EB96E09F938F930E947A0782EB86
:104F400096E00E94E10680918E03282F082E000C27
:104F5000330B3F938F938FEA96E09F938F930E943A
:104F60007A078DEA96E00E94E10680918F03282F50
:104F7000082E000C330B3F938F938AEA96E09F93A1
:104F80008F930E947A0787EA96E00E94E10680915B
:104F90008A031F928F9384EA96E09F938F930E94D7
:104FA0007A0782EA96E00E94E106809189031F92C7
:104FB0008F938FE996E09F938F930E947A078CE9F5
:104FC00096E00E94E1068DB79EB74C960FB6F89416
:104FD0009EBF0FBE8DBF8BE893E00E9438180E94E1
:104FE0000925909388038093870308951F93CF9397
:104FF000DF9380918703909188030E942125AC0163
:1050000090918A03992321F02091270130E006C076
:10501000209128018AE0289F90011124421753070C
:1050200008F485C080918C03C0918D03D0918E03CC
:1050300010918F03811107C0C11175C0D11173C0C8
:10504000111171C074C09F3F19F09F5F90938A0344
:10505000181624F40E94FA2580938C0380918C0307
:1050600087FF05C00E94FA25819580938C031C164A
:1050700024F40E94FA2580938D0380918D0387FF8D
:1050800005C00E94FA25819580938D0360918C0361
:10509000662331F1C0918D03CC2311F1062E000C53
:1050A000770B880B990B0E94A92C23E333E343E38E
:1050B0005FE30E940D2D0E94712C60938C036C2F76
:1050C000CC0F770B880B990B0E94A92C23E333E3B9
:1050D00043E35FE30E940D2D0E94712C60938D03CA
:1050E0001D1624F40E94432680938E0380918E0324
:1050F00087FF05C00E944326819580938E03111679
:1051000024F40E94432680938F0380918F0387FFAE
:1051100005C00E944326819580938F03DF91CF9134
:105120001F910C9469279F3F09F08FCF97CFDF9194
:10513000CF911F910895EBE8F3E085E0DF011D9228
:105140008A95E9F710928A0310928903089586EEF2
:1051500098E00E94E1061F9281E08F931F9285E004
:105160008F9388E998E09F938F930E947A070F901E
:105170000F900F900F900F900F9008958330E9F1EA
:1051800028F4813061F0823009F10895853009F406
:1051900062C008F449C0863009F474C00895809153
:1051A0002801262F30E0280F311D2F3F310524F430
:1051B000680F6093280103C08FEF809328018091CE
:1051C00028011F928F9381ED97E072C08091270193
:1051D000262F30E0280F311D2F3F310524F4680FB2
:1051E0006093270103C08FEF8093270180912701EF
:1051F0001F928F938FEB97E05BC080912601262F43
:1052000030E0280F311D2F3F310524F4680F6093E3
:10521000260103C08FEF80932601809126011F9203
:105220008F938CEA97E044C080912501262F30E0CF
:10523000280F311D2F3F310524F4680F609325019D
:1052400003C08FEF80932501809125011F928F93DA
:1052500087E997E02DC080912401262F30E0280FA8
:10526000311D2F3F310524F4680F6093240103C0E2
:105270008FEF80932401809124011F928F938EE7FA
:1052800097E016C080912301262F30E0280F311DB2
:105290002F3F310524F4680F6093230103C08FEF83
:1052A00080932301809123011F928F9383E697E0DF
:1052B0009F938F930E947A070F900F900F900F90FB
:1052C0000895833081F128F4813059F08230D1F093
:1052D0000895853009F449C0B8F1863009F456C004
:1052E000089580912801681720F4861B8093280177
:1052F00002C010922801809128011F928F9384E5AB
:1053000097E054C080912701681720F4861B809392
:10531000270102C010922701809127011F928F93CD
:1053200082E497E043C080912601681720F4861B31
:105330008093260102C010922601809126011F92BF
:105340008F938FE297E032C080912501681720F497
:10535000861B8093250102C01092250180912501B2
:105360001F928F938AE197E021C0809124016817F2
:1053700020F4861B8093240102C0109224018091A6
:1053800024011F928F9381E097E010C08091230148
:10539000681720F4861B8093230102C0109223011A
:1053A000809123011F928F9386EE96E09F938F93B7
:1053B0000E947A070F900F900F900F900895CF934F
:1053C000C82F1F928F938BEE99E09F938F930E942B
:1053D0007A0781E090E0A0E0B0E0BC01CD0104C01C
:1053E000660F771F881F991FCA95D2F70E94032264
:1053F0000F900F900F900F90CF910C94D21DCF93E0
:10540000873288F58E3108F00BC18E3009F487C0E1
:10541000D8F4873009F460C08B3009F44FC086306F
:1054200009F002C180918103817F8E7F8093810387
:1054300080EF99E00E94E10685EA9CE00E94E10687
:1054400081E08093910346C0863109F4B0C020F416
:10545000803109F47AC0E8C0893109F491C08B31F8
:1054600009F449C0E1C0883349F150F4893209F4A4
:10547000D5C0853309F4D2C0873209F0D5C0CEC07B
:10548000833409F4CBC028F48A3308F4CDC089539F
:10549000C8C0883409F0C8C00E94D21D84E99CE0CD
:1054A0000E94E1062FEF83ED90E321508040904071
:1054B000E1F700C000000E949C250CC087E19AE043
:1054C00041C08BE79CE00E94E106809181038160EE
:1054D00080938103C1E0ADC080918103C82FC1706A
:1054E00080FFEFCF87E89CE00E94E1068091810376
:1054F000817F8E7F3FC09091810391FBCC27C0F9C3
:1055000081E0C827892FC0FB81F980938103CC23D8
:1055100019F08EE69CE029C080E69CE013C09091D3
:10552000810392FBCC27C0F981E0C827892FC0FBFB
:1055300082F980938103CC2319F081E59CE015C0AA
:1055400081E49CE00E94E106C5CF9091810393FB2A
:10555000CC27C0F981E0C827892FC0FB83F980934D
:105560008103CC2351F085E39CE00E94E106809109
:1055700081038160809381035CC088E29CE0E2CF7C
:1055800089E19CE00E94E1068CEE9BE00E94E1062E
:1055900085EB9BE00E94E10688E89BE00E94E10623
:1055A00083E49BE00E94E10685E19BE0CBCF87E0AE
:1055B0009BE00E94E1060E94E3171F928F938DEEFD
:1055C0009AE09F938F930E947A07809120011F9207
:1055D0008F9386ED9AE09F938F930E947A07809134
:1055E000E4021F928F9383EC9AE09F938F930E9423
:1055F0007A070E9415259F938F937F936F938CEA70
:105600009AE09F938F930E947A078DB79EB7429638
:105610000FB6F8949EBF0FBE8DBF5CCF80E001C077
:105620008D510E94DF2956CF8AEA9AE00E94E10656
:10563000C0E08C2FCF910895CF93C82F8091910314
:10564000813071F020F0823009F44BC042C1E0910A
:105650002101F09122018081823209F03CC107C012
:10566000E0912101F09122018081823261F48C2F3E
:105670000E94D20B811104C08C2F0E94FF292FC0E1
:1056800081E090E02CC08C2F0E94FF0D811126C07C
:10569000C431E1F070F4CB3081F0C031D1F40E941C
:1056A000A72883EE99E00E94E10682E080939103AF
:1056B00015C0C93259F0C83361F480EF99E00E94F7
:1056C000E10687EE99E00E94E10608C0109291037E
:1056D00004C181EE99E00E94E106FFC081E0817083
:1056E000FEC0C43228F5CE3108F0C1C0CB30A1F1E4
:1056F000D0F4C73009F0D3C08EE18093280182E353
:10570000809327018AE08093260184E1809325011C
:1057100088E08093240188E28093230187E898E061
:105720000E94E106BFC0C33149F1C431C1F0B7C026
:10573000CB3409F4A9C028F4C93289F0C83361F028
:10574000AEC0C13509F49EC0C23509F499C0CE344B
:1057500009F0A5C06AE09EC00E94A728A3C080915E
:105760009003882319F0109290039CC084E998E07C
:105770000E94E10681E080939103B1C08EE698E03B
:105780000E94E1068CE598E00E94E10680912801E4
:105790001F928F9389E598E09F938F930E947A07D9
:1057A00087E598E00E94E10685E498E00E94E10622
:1057B000809127011F928F9382E498E09F938F93AB
:1057C0000E947A0780E498E00E94E10681E398E075
:1057D0000E94E106809126011F928F938EE298E04D
:1057E0009F938F930E947A078CE298E00E94E106D3
:1057F0008BE198E00E94E106809125011F928F9332
:1058000088E198E09F938F930E947A0786E198E061
:105810000E94E10681E098E00E94E1068091240167
:105820001F928F938EEF97E09F938F930E947A073A
:105830008CEF97E00E94E10685EE97E00E94E1067A
:10584000809123011F928F9382EE97E09F938F9315
:105850000E947A0780EE97E00E94E1068DB79EB71E
:1058600048960FB6F8949EBF0FBE8DBF1BC0CE5199
:10587000EC2FF0E0E057FE4F80818093900312C040
:1058800061E003C061E006C06AE0809190030E947D
:10589000BE2808C0809190030E94612903C085E85A
:1058A00098E013C080919003882369F01F928F9332
:1058B0008FE798E09F938F930E947A070F900F9045
:1058C0000F900F9004C08CE798E00E94E10681E001
:1058D00006C01092910380E002C080E000CFCF911B
:1058E00008950E94782C6894B1110C94072D0895A6
:1058F0000E94EC2C88F09F5798F0B92F9927B75148
:10590000B0F0E1F0660F771F881F991F1AF0BA9563
:10591000C9F714C0B13091F00E94062DB1E008958E
:105920000C94062D672F782F8827B85F39F0B93F80
:10593000CCF3869577956795B395D9F73EF4909516
:105940008095709561957F4F8F4F9F4F0895E89494
:1059500009C097FB3EF490958095709561957F4FB7
:105960008F4F9F4F9923A9F0F92F96E9BB27939565
:10597000F695879577956795B795F111F8CFFAF475
:10598000BB0F11F460FF1BC06F5F7F4F8F4F9F4FA6
:1059900016C0882311F096E911C0772321F09EE804
:1059A000872F762F05C0662371F096E8862F70E06A
:1059B00060E02AF09A95660F771F881FDAF7880F44
:1059C0009695879597F9089557FD9058440F551F60
:1059D00059F05F3F71F04795880F97FB991F61F071
:1059E0009F3F79F087950895121613061406551FE8
:1059F000F2CF4695F1DF08C0161617061806991F54
:105A0000F1CF86957105610508940895E894BB2748
:105A100066277727CB0197F908950E94202D0C94D3
:105A2000912D0E94832D38F00E948A2D20F095231D
:105A300011F00C947A2D0C94802D11240C94072DC8
:105A40000E94E42C70F3959FC1F3950F50E0551F11
:105A5000629FF001729FBB27F00DB11D639FAA27C3
:105A6000F00DB11DAA1F649F6627B00DA11D661F12
:105A7000829F2227B00DA11D621F739FB00DA11D33
:105A8000621F839FA00D611D221F749F3327A00DED
:105A9000611D231F849F600D211D822F762F6A2F89
:105AA00011249F5750409AF0F1F088234AF0EE0FEE
:105AB000FF1FBB1F661F771F881F91505040A9F71B
:105AC0009E3F510580F00C947A2D0C94072D5F3F7A
:105AD000E4F3983ED4F3869577956795B795F79557
:105AE000E7959F5FC1F7FE2B880F911D96958795CF
:105AF00097F9089597F99F6780E870E060E008954E
:105B00009FEF80EC089500240A94161617061806D5
:105B10000906089500240A941216130614060506B1
:105B20000895092E0394000C11F4882352F0BB0F42
:105B300040F4BF2B11F460FF04C06F5F7F4F8F4FA5
:105B40009F4F0895991B79E004C0991F961708F09C
:105B5000961B881F7A95C9F780950895AA1BBB1BD1
:105B600051E107C0AA1FBB1FA617B70710F0A61B5D
:105B7000B70B881F991F5A95A9F780959095BC017E
:105B8000CD01089597FB072E16F4009407D077FDFA
:105B900009D00E94AE2D07FC05D03EF4909581956A
:105BA0009F4F0895709561957F4F0895A1E21A2E39
:105BB000AA1BBB1BFD010DC0AA1FBB1FEE1FFF1FB1
:105BC000A217B307E407F50720F0A21BB30BE40B01
:105BD000F50B661F771F881F991F1A9469F7609548
:105BE0007095809590959B01AC01BD01CF01089502
:105BF000EE0FFF1F0590F491E02D0994F894FFCF6C
:105C000027092A092B092C092D092309A7098D0920
:105C100026092E090A019C108D116A1136110211F4
:105C20000177032808140A321E524E2D3432004CDC
:105C3000554641004F4646004F4E00434F4E4E00E2
:105C4000506F776572656400556E61747461636846
:105C500065640044656661756C74004164647265D6
:105C60007373656400436F6E66696775726564007F
:105C70003F0053757370656E64656400404D362255
:105C8000F205A5056F054D05D904F2040B052405A1
:0A5C900001020304050607080900DD
:106800000000000000000000040005000600070072
:10681000080009000A000B000C000D000E000F001C
:1068200010001100120013001400150016001700CC
:10683000180019001A001B001C001D001E001F007C
:10684000200021002200230024002500260027002C
:106850002800000035002B002C002D002E002F00FA
:1068600030002A00000033003400290036003700D1
:106870003800E00000000000000000000000000000
:106880000000000000000000000000000000000008
:1068900000000000000000000000000000000000F8
:1068A00000000000000000000000000000000000E8
:1068B00000000000000000000000000000000000D8
:1068C00000000000000000000000000000000000C8
:1068D00000000000000000000000000000000000B8
:1068E0000000000000000000310000000000000077
:1068F0000000E100E200E300F1A1E500E600E700AE
:106900000000000000000000EA4401000100E24431
:106910000100010001005500460054004A004B00F0
:10692000560057004700480001000100E9440100FB
:106930000100010001000100010001003A003B00DC
:106940003C003D003E003F0040004100420043004B
:10695000580000004C00390001004400450052007E
:1069600001000100000050004F0081404D004E002A
:1069700051000100000000000000000000000000C5
:106980000000000000000000000000000000000007
:1069900000000000000000000000000000000000F7
:1069A00000000000000000000000000000000000E7
:1069B00000000000000000000000000000000000D7
:1069C00000000000000000000000000000000000C7
:1069D00000000000000000000000000000000000B7
:1069E000000000000000000049000000000000005E
:1069F0000000010001000100010001000100010090
:00000001FF
